:100000000C9475000C94EB010C9492000C949200EB
:100010000C9492000C9492000C9492000C94920018
:100020000C9492000C9492000C9492000C94920008
:100030000C9492000C9492000C9492000C949200F8
:100040000C9492000C9492000C9492000C949200E8
:100050000C9492000C9492000C9492000C949200D8
:100060000C9492000C9492001E0332006100780000
:100070006500730031003600620075007400740082
:100080006F006E007300180372006100700068005A
:100090006E00650074002E006E006500740004039D
:1000A00009040A0331003000300038000501090559
:1000B000A1010901A10009300931150026FF0075D1
:1000C0000895028102C005091901291015002501B2
:1000D000750195108102C012010101000000088124
:1000E000179C0A0201010203010011241FBECFEF79
:1000F000D4E0DEBFCDBF11E0A0E0B1E0E8E0FBE07E
:1001000002C005900D92A23EB107D9F722E0A2EEFF
:10011000B1E001C01D92A133B207E1F70E94D10402
:100120000C9482050C940000CF93C62F20910001FF
:1001300024FF0BC02091070238E8232720930702F1
:10014000FC01A8E0B2E08C2F04C02AE52093000156
:10015000F7CF815018F091919D93FBCF6C2F88E0E1
:1001600092E00E94E701CC5FC0930001CF91089517
:10017000CF93DF938091170218160CF0AEC09091C8
:100180001402209113022D3219F090E880E09FC0F4
:100190002AE5209301018B30C1F7CCE0D0E0C91BE8
:1001A000D109C55EDD4F8881807609F080C010924C
:1001B0000502898181110BC01092060285E092E050
:1001C000909316028093150290E882E079C0853002
:1001D00021F48A818093180271C0863009F04BC0E7
:1001E0008B81813009F442C0823021F4CE010E941B
:1001F0004E0360C0833069F58A81811109C08EE9A0
:1002000090E0909316028093150290EC84E058C021
:10021000813049F486E890E09093160280931502AD
:1002200090EC88E14DC0823049F488E690E09093EC
:1002300016028093150290EC8EE142C08330E1F506
:1002400082EA90E0909316028093150290EC8CE085
:1002500037C0813249F485EF91E090931602809384
:10026000150290EC89E02CC0823231F5CE010E945B
:100270004E0390EC25C0883019F48AE192E00AC060
:10028000893021F48A8180931A0218C08A3049F497
:1002900085E092E0909316028093150290E881E049
:1002A0000FC08B3059F483EC8093070207C0CE0156
:1002B0000E947C0390E804C090EC01C090E880E0CC
:1002C0002F81211104C02E81281708F4822F9093CA
:1002D000E20180930201109217028091010184FFD4
:1002E00046C0809102018F3F09F441C0C82F893078
:1002F00008F0C8E08C1B809302012091E20120FDF0
:1003000002C0DBE401C0D3EC2F5F2093E2018091B7
:1003100015029091160226FD05C0FC01ADEFB1E07B
:100320002C2F0AC0ADEFB1E0FC012C2F215048F07A
:1003300034913D933196FACF215018F031913D938D
:10034000FBCF8C0F911D90931602809315026C2F9A
:100350008DEF91E00E94E70184E08C0FC83019F026
:100360009FEF90930201D093FC01809301018AE0FA
:1003700099B1957031F48150D9F71092180210920A
:100380001202DF91CF910895E9E6F0E08081836069
:100390008083E89A83EC809307020895A82FB92FF1
:1003A0008FEF9FEF41E050EA615070F02D9138E0FF
:1003B000722F782796958795269570FF02C084271F
:1003C00095273A95A9F7F0CF809590950895E6DFA7
:1003D0008D939D930895CF93CFB7CF93489BFECF36
:1003E000489B09C0489B07C0489B05C0489B03C069
:1003F000489B01C09EC0DF93C0911402DD27C55EFB
:10040000DD4F489B02C0DF91EBCF2F930F931F93DB
:1004100009B12FEF00FB20F94F933F9319B14FEF34
:10042000012700FB21F93BE031C04E7F012F19B1BC
:10043000216028C0102F4D7F2260000009B129C023
:100440004B7F2460012F000019B12BC019B1477FE9
:1004500028602AC04F7E09B120612CC04F7D19B1A0
:1004600020622FC04F7B09B1206432C0422709B1FE
:1004700049934FEF0000102710FB20F919B11570B8
:10048000A9F1297F91F2012700FB21F909B1237F0E
:1004900089F23150F0F1102710FB22F919B1277EB3
:1004A00079F2012700FB23F92F7C81F209B1102793
:1004B00010FB24F92F7971F200C019B1012700FB5C
:1004C00025F92F7359F200C009B1102710FB26F946
:1004D000223040F200C019B1012700FB27F9243077
:1004E00028F64F77206819B10000F9CF3B503195BD
:1004F000333011E01CBBB8F0C31BD0400881033C73
:1005000041F10B3431F11981412F1F7720911202F3
:10051000121731F4093691F10D3279F0013E69F08C
:100520002227209319023F914F911F910F912F91F4
:10053000DF91CF91CFBFCF911895009319023F91D2
:100540004F911F910F912F91DF91CCB3C0FD46CFFA
:10055000F0CF00911902002331F3109117021123FB
:10056000A1F53430A2F130931702009313021091D9
:1005700014023BE0311B3093140229C00091170292
:1005800001301CF50AE547FD09C03091010134FD39
:1005900020C000930101CCEFD1E01FC030910001D9
:1005A00034FD17C000930001C7E0D2E016C0052754
:1005B00010E00BB91FC0052722C0052727C005275B
:1005C0002CC0052710E00BB933C04AE503C042ED4B
:1005D00001C0432FC4E1D0E032E01AB11560589A4F
:1005E0000BB11AB95F9355E020E820FF05270BB93E
:1005F000279517951C3FD8F620FF052727950BB99F
:1006000017951C3FC0F620FF0527279517950BB9B6
:100610001C3F98F620FF0527279517951C3F0BB91F
:1006200070F600C0499120FF05270BB92795179553
:100630001C3F38F620FF052727950BB917951C3F5F
:1006400038F520FF0527279517950BB91C3F10F5A6
:1006500020FF0527279517951C3F0BB9E8F4242F99
:100660003A9519F60A7F5F910BB900C010911802F4
:10067000C651D04011F01093120211E01CBB016072
:100680001AB11A7F402F4A7F0BB91AB94BB94BCF19
:100690000527D3CF0527D8CF0527DDCFFC018081E3
:1006A000807641F59181963031F593819230D1F089
:1006B000923269F09130F9F48091ED019091EE0160
:1006C00090931602809315028091EC010895809119
:1006D000F0019091F10190931602809315028091A0
:1006E000EF01089583E091E0909316028093150244
:1006F00082E2089580E0089524EE31E030931602FE
:1007000020931502FC0120812076203299F481810A
:10071000813081F4E091EA01F091EB010088F189E8
:10072000E02D84EE91E00995E091EA01F091EB0172
:100730008081089580E00895009769F04091F80164
:100740005091F9016091FA017091FB01FC01408325
:100750005183628373838091F8019091F901A09194
:10076000FA01B091FB018093F4019093F501A093FD
:10077000F601B093F701089524B1217C24B925B185
:100780002E6325B918B820E227B92FE128B9E7EB85
:10079000FBE03197F1F700C0000026B120952F71E2
:1007A0002A3150F430E0F901E853FE4F4081F9015D
:1007B000E255FE4F208102C020E040E0FC01408372
:1007C000FB01208308950F931F93CF93DF9300D0F5
:1007D00000D0CDB7DEB7BE016F5F7F4FCE0102966E
:1007E0000E94BC0387B1817E87B988B18E6188B9C8
:1007F00085B1877C85B984B1886384B987EB9BE038
:100800000197F1F700C0000026B1269588B1817EDE
:1008100088B987B18E6187B985B1877C85B984B184
:10082000877C84B985B1886385B987EB9BE00197A4
:10083000F1F700C0000083B1869586958695809576
:100840002095877030E1839FC00111242F70822B87
:1008500041978833910540F4FC01EE0FFF1FE25CE5
:10086000FE4F0081118102C000E010E018B817B8F7
:100870008FEF88B915B888E084B985B1806385B9F0
:1008800087EB9BE00197F1F700C0000083B184FF84
:10089000046085FF016015B880E184B92D9A87EB6B
:1008A0009BE00197F1F700C000001D9B0260C801AA
:1008B000887F892B21F08091F3018C8315C0BE01C4
:1008C0006D5F7F4FCE0104960E94BC038C819A819C
:1008D000891721F08091F3018C8302C08093F3018A
:1008E0008B819981891721F08091F2018B8302C05D
:1008F0008093F2019C818FE3989F902D1124905852
:100900009093F8019B81989F802D112480588093AB
:10091000F9010093FA011093FB010F900F900F90D3
:100920000F90DF91CF911F910F910895CF93CFB783
:10093000F89417B814B88FEF88B985B90E94E3030B
:10094000CFBFCF9108958091250190912601892BE9
:1009500031F0109226011092250181E0089544E0C3
:1009600050E064EF71E088EF91E00E947505089512
:100970008E5F853038F4E82FF0E0E75CFE4F808131
:1009800090E0089580E890E008958CEA90E09093DC
:100990002C0180932B0187E291E0089582E190E0A1
:1009A000089581E084B98EEF85B917B88FEF88B9C3
:1009B00088EF8BB985E08AB982E08093B00087E048
:1009C0008093B10084EC8093B300209A84B1897F36
:1009D00084B985B1866085B928980E94C504FC0158
:1009E0009093EB018093EA01848195819093F101CA
:1009F0008093F00182818093EF018085918500973B
:100A000031F09093EE018093ED01868108C087ED6F
:100A100090E09093EE018093ED010E94CE048093CC
:100A2000EC018091EF0180931C018BB18A7F8BB91F
:100A30008AB185608AB987EC9FEA0197F1F700C017
:100A400000008AB18A7F8AB9E091EA01F091EB0156
:100A50000284F385E02D09950E94C401789411E089
:100A6000D0E0C2E0A8950E94B800112341F0E091C7
:100A7000EA01F091EB010484F585E02D0995B99B1D
:100A800016C0C7BBD11115C0E091EA01F091EB018E
:100A90000484F585E02D0995E091EA01F091EB01E0
:100AA0000684F785E02D0995811103C01CC0DD2364
:100AB000D1F08091000184FD03C0D1E010E0D2CFDD
:100AC000E091EA01F091EB010088F189E02D84EEDC
:100AD00091E00995E091EA01F091EB01608184EEEB
:100AE00091E00E949400D0E0E9CFFB01DC0104C05A
:100AF0008D910190801921F441505040C8F7881B16
:080B0000990B0895F894FFCF52
:100B08005A5AFF090222000101008032090400003C
:100B1800010300000009210101000122000007056E
:100B2800810308000A010004002B000000000000F7
:100B3800009604E303A3049C03004080C0FF001058
:100B48000002000040000000000000000800000053
:100B5800000000000000000000000000000000206D
:100B680000040000800000000000000010000000E9
:100B7800000000000000000000000000000000006D
:100B8800000000000000000000000000000000005D
:100B9800000000000000000000000000000000400D
:100BA8000008000000010000000000002000000014
:100BB80000FFFEFEFEFE00010000FFFE0000020234
:100BC80001020000000002020000FEFE0001FFFE1C
:100BD800020200000202000000FFFEFE000000000A
:020BE800010208
:00000001FF
